:100000000C949B050C94D3050C94D3050C94D30548
:100010000C94D3050C94D3050C94D3050C94D30500
:100020000C94D3050C94D3050C9426280C94F82832
:100030000C945C220C94D3050C94D3050C94D3053A
:100040000C94D3050C94D3050C94D3050C94D305D0
:100050000C94D3050C94E4220C94D3050C94D30592
:100060000C94D3050C94D3050C94D3050C94D305B0
:100070000C94D3050C94D3050C94D3050C94D305A0
:100080000C94D3050C94D3050C94D3050C94D30590
:100090000C94D3050C94D3050C94D3050C94D30580
:1000A0000C94D3050C94D3050C94D305690B690B00
:1000B000950B950BFD0B1B0C330D330D260CBF0C54
:1000C000D00CD00C65298C29842A8C29842AD82923
:1000D000FB29842A522A612A7467670074676C6856
:1000E0006600AD43A900AE00AC00AA00AB002943F6
:1000F0001D011D031B01060119011E431F002000E5
:100100002100A75DA85D01000100005C10501150A6
:100110001250010001000100010001000100010076
:1001200001000100010001000100010001000100C7
:1001300001000100010001000100010001000100B7
:1001400001000100010001000100010001000100A7
:100150000100010001000100010001000100010097
:100160000100010001000100010001000100010087
:100170000100010001000100010001000100010077
:100180000100010001000100010001000100010067
:100190000100010001000100010001000100010057
:1001A000010044454255473A2064697361626C65B9
:1001B000642E0A0044454255473A20656E61626CE0
:1001C00065642E0A0000000000000000002A2B28B1
:1001D000000000000000000000000000000000001F
:1001E00029000000002C1E3420212224342627253B
:1001F0002E362D3738271E1F202122232425263373
:1002000033362E37381F0405060708090A0B0C0D74
:100210000E0F101112131415161718191A1B1C1D86
:100220002F3130232D350405060708090A0B0C0D64
:100230000E0F101112131415161718191A1B1C1D66
:100240002F3130354C00000000000000000000009D
:10025000000000000000000000000000000000009E
:100260000000000000000000007E0F00D4FFFFFF30
:10027000C7000000780A0025303258006C65645FC2
:100280007461736B3A20004F6E6573686F743A2027
:100290006163746976653A2025640A000A00253096
:1002A0003862003A200025303258000A722F63204D
:1002B00030313233343536370A00290A00257500CB
:1002C0002F002575005D28002564002000256400AE
:1002D000200025640020002564007C002530325871
:1002E000006D6F7573656B6579205B62746E7C78E9
:1002F0002079207620685D287265702F61636C29F3
:100300003A205B00313A0964656C6179282A313002
:100310006D73293A2025750A323A09696E7465723F
:1003200076616C286D73293A2025750A333A096D78
:1003300061785F73706565643A2025750A343A09FF
:1003400074696D655F746F5F6D61783A2025750A19
:10035000353A09776865656C5F6D61785F737065C4
:1003600065643A2025750A363A09776865656C5FD9
:1003700074696D655F746F5F6D61783A2025750AE9
:1003800000703A097072696E742076616C756573DD
:100390000A643A097365742064656661756C7473E8
:1003A0000A75703A092B310A646E3A092D310A6CCC
:1003B000743A092B31300A72743A092D31300A45EA
:1003C00053432F713A09717569740A0A7370656530
:1003D00064203D2064656C7461202A206D61785F23
:1003E0007370656564202A202872657065617420C9
:1003F0002F2074696D655F746F5F6D6178290A776E
:10040000686572652064656C74613A206375727307
:100410006F723D25642C20776865656C3D25640A04
:1004200053656520687474703A2F2F656E2E776956
:100430006B6970656469612E6F72672F77696B698C
:100440002F4D6F7573655F6B6579730A004D3E20A4
:10045000004D25753A25733E20003F0A003D2025BA
:10046000750A003F0A0064656661756C74730A0062
:1004700025750A003F0A000A092D2056616C756532
:1004800073202D0A00710A000A092D204D6F757323
:10049000656B6579202D0A003F00433E20004C2506
:1004A000640A000A092D20537461747573202D0AA3
:1004B000686F73745F6B6579626F6172645F6C659E
:1004C000647328293A20253032580A6B6579626FA7
:1004D0006172645F70726F746F636F6C3A20253065
:1004E00032580A6B6579626F6172645F69646C652A
:1004F0003A20253032580A74696D65725F72656101
:1005000064333228293A202530386C580A000A0909
:100510002D2056657273696F6E202D0A5649443A34
:100520002030784645464428416C6C74726F6E7377
:1005300020495429205049443A2030783934363003
:10054000284B6E6F7073204D696E69292056455295
:100550003A203078303030310A4255494C443A2004
:1005600020284665622032372032303232290A4F45
:100570005054494F4E533A204C554641204D4F550B
:1005800053454B45592045585452414B45592043FA
:100590004F4E534F4C4520434F4D4D414E44203418
:1005A0003039360A4743433A20352E342E30204125
:1005B00056522D4C4942433A20322E302E302041A3
:1005C00056525F415243483A20617672350A000A1A
:1005D000092D20436F6E736F6C65202D0A455343C0
:1005E0002F713A09717569740A6D3A096D6F7573E7
:1005F000656B65790A000A092D204D6167696320E2
:100600002D0A443A094465627567204D657373612C
:10061000676520546F67676C650A583A094D6174C5
:10062000726978204465627567204D6F6465205457
:100630006F67676C65202D2053686F77206B657935
:100640007072657373657320696E206D6174726971
:100650007820677269640A4B3A094B6579626F6169
:10066000726420446562756720546F67676C65200B
:100670002D2053686F77206B6579707265737320D6
:100680007265706F72740A4D3A094465627567202D
:100690004D6F75736520546F67676C650A563A092C
:1006A00056657273696F6E0A533A095374617475B3
:1006B000730A433A09416374697661746520436F34
:1006C0006E736F6C65204D6F64650A46312D46313F
:1006D000303A0953776974636820746F204C6179EC
:1006E000657220302D392028463130203D204C3095
:1006F000290A302D393A0953776974636820746F79
:10070000204C6179657220302D390A475241564597
:100710003A0953776974636820746F204C61796576
:100720007220302028616C7465726E617465290ACC
:10073000423A094A756D7020746F20426F6F746C75
:100740006F616465720A4553433A094A756D7020BA
:10075000746F20426F6F746C6F61646572202861E2
:100760006C7465726E617465290A453A0950726944
:100770006E7420454550524F4D2053657474696E18
:1007800067730A4253504143453A09436C656172AD
:1007900020454550524F4D0A006B65796D61705F81
:1007A000636F6E6669672E7261773A202530325822
:1007B0000A2E737761705F636F6E74726F6C5F6324
:1007C0006170736C6F636B3A2025750A2E636170DC
:1007D000736C6F636B5F746F5F636F6E74726F6C5B
:1007E0003A2025750A2E737761705F6C63746C5FB5
:1007F0006C6775693A2025750A2E737761705F7290
:1008000063746C5F726775693A2025750A2E737779
:1008100061705F6C616C745F6C6775693A202575F7
:100820000A2E737761705F72616C745F72677569AD
:100830003A2025750A2E6E6F5F6775693A20257517
:100840000A2E737761705F67726176655F657363A7
:100850003A2025750A2E737761705F6261636B734E
:100860006C6173685F6261636B73706163653A208A
:1008700025750A2E6E6B726F3A2025750A00646525
:100880006275675F636F6E6669672E7261773A2083
:10089000253032580A2E656E61626C653A202575E6
:1008A0000A2E6D61747269783A2025750A2E6B657F
:1008B00079626F6172643A2025750A2E6D6F7573C7
:1008C000653A2025750A006565636F6E6669673A4B
:1008D0000A64656661756C745F6C617965723A2053
:1008E00025750A003F000A6D6F7573653A206F66C3
:1008F000660A000A6D6F7573653A206F6E0A000A0A
:100900006B6579626F6172643A206F66660A000AED
:100910006B6579626F6172643A206F6E0A000A6DCE
:1009200061747269783A206F66660A000A6D6174B4
:100930007269783A206F6E0A000A64656275673AD8
:10094000206F66660A000A64656275673A206F6EFA
:100950000A000A0A4A756D70696E6720746F20621A
:100960006F6F746C6F616465722E2E2E2000433E93
:100970002000436C656172696E6720454550524F97
:100980004D0A000A002530325820006B6579626FED
:100990006172645F7265706F72743A20005B735DA0
:1009A000005B575D005B535D005B525D005B445D27
:1009B000005B435D0016034B006E006F0070007318
:1009C0000020004D0069006E00690000001803411E
:1009D000006C006C00740072006F006E00730020E9
:1009E000004900540000000403090409025B0003ED
:1009F0000100A0FA0904000001030101000921110E
:100A000001000122400007058103080001090401DB
:100A1000000103000000092111010001227B0007F1
:100A200005820320000109040200020300000009FE
:100A30002111010001222200070583032000010784
:100A40000503032000011201000200000008FDFE62
:100A500060940100010200010631FF0974A101093F
:100A600075150026FF00952075088102097615008E
:100A700026FF00952075089102C005010902A10119
:100A800085020901A10005091901290815002501A0
:100A90009508750181020501093009311581257F0D
:100AA00095027508810609381581257F950175081D
:100AB0008106050C0A38021581257F95017508818C
:100AC00006C0C005010980A101850319012AB700EC
:100AD000150126B700950175108100C0050C0901AC
:100AE000A101850419012AA002150126A002950181
:100AF00075108100C005010906A101050719E0294B
:100B0000E715002501950875018102950175088199
:100B1000010507190029FF150026FF009506750835
:100B200081000508190129059505750191029501B6
:100B300075039101C00011241FBECFEFDAE0DEBFC4
:100B4000CDBF04B603FE18C080919C0290919D0217
:100B5000A0919E02B0919F028730904BA740B04B6E
:100B600059F410929C0210929D0210929E021092D3
:100B70009F02E0E0F8E3099511E0A0E0B1E0E4E8CD
:100B8000F6E502C005900D92AE3EB107D9F722E01E
:100B9000AEEEB1E001C01D92AC39B207E1F70E94A0
:100BA000B9180C94402B0C940000FF93EF93E09144
:100BB000EE01F091EF01309709F00995EF91FF9167
:100BC0000895FC018591803011F0EFDFFBCF08958F
:100BD000FF27E0E230E247FF0CC0419597FF09C0D4
:100BE000EDE26095709580959095611D711D811D58
:100BF000911D27FF02C0219530E350E2AA27660F1E
:100C0000771F881F991FAA1FA41710F0A41B6395B4
:100C10005A95A9F7AA3008F0A95FA05DAF93F395A4
:100C2000611571058105910541F7ED3211F4EF93DE
:100C3000F395F21718F43F93F395FBCF8F91B5DF3F
:100C4000FA95E1F70895E991F9918591803021F0C5
:100C5000853219F0AADFF9CF089520E0E894559184
:100C60005532C1F3503311F4689455915A3348F416
:100C7000505390F3220F022E220F220F200D250F2A
:100C8000F4CF0EF4219589919991533619F3533786
:100C900029F1533559F1BC0188279927E8945C362E
:100CA00021F48991999168945591543639F446EF1D
:100CB0007EF077FF0DC08FEF9FEF0AC055374AE0F7
:100CC00039F0583540E121F0523642E009F00895FC
:100CD000FF93EF937DDFEF91FF91B7CFFF93EF93FA
:100CE000FC0181918030B9F360DFFBCFFF93EF937C
:100CF00068DFF1CFDF93CF93CDB7DEB72596A3DFC3
:100D0000CF91DF910895662309F183309105B1F009
:100D100034F48130910551F0029751F008958530F7
:100D2000910581F06CF0069779F008955F9A089527
:100D30001F9B02C0469A0895479A08955C9A0895A9
:100D4000769A08952C9A08955E9A089583309105B5
:100D5000B1F034F48130910551F0029751F00895CB
:100D60008530910581F06CF0069779F008955F98D1
:100D700008951F9B02C046980895479808955C986F
:100D80000895769808952C9808955E9808955D9A30
:100D90002E98289A8130910539F08230910531F0F2
:100DA000892B29F45D9808952E9A0895289808951E
:100DB000579A5F983E9A3F9A46984798549A5C98FB
:100DC0006E9A7698249A2C98569A5E98559A269AF6
:100DD000209A08950E94D8062F9A27985F9A469ADB
:100DE000479A5C9A769A2C9A5E9A80E090E00C94EE
:100DF000C7068130910531F18230910509F444C074
:100E0000892B09F045C080E090E00E94C70661E0B0
:100E100081E090E00E94830661E082E090E00E9421
:100E2000830661E083E090E00E94830661E084E055
:100E300090E00E94830661E085E090E00E948306D6
:100E400061E01EC081E090E00E94C70660E081E0A2
:100E500090E00E94830660E082E090E00E948306BA
:100E600060E083E090E00E94830660E084E090E030
:100E70000E94830660E085E090E00E94830660E0C7
:100E800086E090E00C94830682E090E00C94C70624
:100E90000895CF93FB01823120E59207E9F040F4F9
:100EA000803120E5920761F08131904579F02EC0C4
:100EB000873A2DE59207C1F0883A9D45D9F026C0C2
:100EC000C281CC2319F180E090E00BC0C281CC2319
:100ED000E9F081E090E005C0C281CC23B9F082E066
:100EE00090E00E94F90613C0C281CC2381F08CED02
:100EF00090E005C0C281CC2351F088ED90E00E94C3
:100F00003A0988E20E94170BC0E001C0C1E08C2FB3
:100F1000CF91089581E008950C94490708950C94A9
:100F20008E071F93CF93DF9300D000D01F92CDB7D1
:100F3000DEB749835A836B833091F10189819A81AD
:100F4000311114C0662359F0222349F00E94720F18
:100F5000182F682F89819A810E94190F03C00E945F
:100F6000450F182F69817A81812F04C00E94720F6A
:100F700069817A810F900F900F900F900F90DF9101
:100F8000CF911F910C948716FC01262F408151812F
:100F90006281738184810C94910781E00895CF93DD
:100FA000DF93EC0160E00E94C407BE01DF91CF91A6
:100FB0000C948F070C94D6170C94D41708950E94A4
:100FC000C30D0E94DE072FEF84E39CE02150804098
:100FD0009040E1F700C000000C940A230F931F9388
:100FE000CF93DF938C0161E00E94C407EC01B8014C
:100FF0000E948C07882309F45BC0B801CE010E94CF
:10100000EF20882309F454C0B801CE010E94D11BFF
:10101000882309F44DC0B801CE010E944B208823DB
:1010200009F446C0F80182818823D9F1CF3D8CE5CF
:10103000D80779F140F4C115FCE5DF0791F0C13024
:10104000DC4591F02EC0CC35EDE5DE0741F1CD3524
:10105000FDE5DF0709F1CB35DD4519F50E940914DF
:1010600020C00E94DF0724C080915402C82FC09581
:10107000C170C0FB80F980935402CC2329F084EB2B
:1010800091E00E94E10514C082EA91E00E94E1052E
:1010900010C00E94B7140CC00E94001402C00E942D
:1010A0000C14C801DF91CF911F910F910C948A0706
:1010B000C0E08C2FDF91CF911F910F9108950E9476
:1010C00044220C9460090E9463090C944A22DF9226
:1010D000EF92FF920F931F93CF93DF93E82FF0E0EF
:1010E000EB53FE4FD490282F26952695269530E079
:1010F000F901EB59FD4F0491877010E0082E02C0F2
:10110000159507950A94E2F701701127F901EB5A3A
:10111000FD4FE490F12C082E02C0F594E7940A9458
:10112000E2F791E0E922FF24F901EB5BFD4FC49166
:10113000D0E002C0D595C7958A95E2F7C170DD274A
:101140000115110519F081EE0E94E909E114F1047D
:1011500019F086EE0E94E9098D2D0E94170BEF28E9
:1011600019F086EE0E94980A012B19F081EE0E9478
:10117000980ACD2B51F08CE2DF91CF911F910F9106
:10118000FF90EF90DF900C94170BDF91CF911F91A0
:101190000F91FF90EF90DF900895EF92FF920F93E1
:1011A0001F93CF93DF938C01F62E8AE0E82EF8018F
:1011B0008491882309F457C0813009F042C0E801C6
:1011C0002196FE018491813031F42196FE018491B3
:1011D0000E94170B39C0823039F4E8012296FE01D3
:1011E00084910E94E90930C0833039F4E8012296E5
:1011F000FE0184910E94980A27C0843029F5E801F5
:101200002296FE01249180E090E030E020533109E5
:101210002A30310560F4E89EA001E99E500D1124AA
:10122000C901840F951F2196FE012491EECF0097EE
:1012300059F0EFE9FFE03197F1F700C000000197A6
:10124000F6CF0E946708E8018E010F5F1F4F8F2DB8
:10125000882309F4ACCFEFE9FFE03197F1F700C044
:1012600000008150F5CFDF91CF911F910F91FF903A
:10127000EF90089560E00C94CD088295982F9373B9
:1012800044E0949F900111248C7C86958695282BB0
:10129000822F8575880F2A7A2695822B08950895C6
:1012A0000C944F0981E008950C9452090895CF934E
:1012B000C82F0E9450098C2F0E945409CF91089585
:1012C00080E00C9457090E944B210C945709CF934E
:1012D0000E944B21C82F8091F001C81741F1C093A3
:1012E000F0018091540282FF1EC080FF04C08CE791
:1012F00092E00E94E1058091540280FF0CC01F9291
:10130000CF9387E792E09F938F930E947A060F9086
:101310000F900F900F908091540280FF04C085E7DA
:1013200092E00E94E1058C2FCF910C945709CF9148
:101330000895CF93DF93CDB7DEB72B970FB6F89410
:10134000DEBF0FBECDBF4F83588769877A878B87F3
:1013500061110E9438139E012F5F3F4F86E0F90113
:1013600011928A95E9F785E0FE013796D90101903F
:101370000D928A95E1F789819A814C815D81452B97
:1013800031F09F3F31F491E08F3F19F403C091E0B9
:1013900001C090E090FF09C049815A816B817C8136
:1013A0008D819E810E94591205C0C9010E94CD07FE
:1013B0008111F2CF2B960FB6F894DEBF0FBECDBFD2
:1013C000DF91CF910895FC01808191810E94B40F3B
:1013D0000895CF93882309F4A9C0C82F8238C1F497
:1013E0000E944B2181FDA2C069E38091020190918E
:1013F00003010E941C220E945A132FEF81EE94E0F9
:10140000215080409040E1F700C0000069E319C01E
:10141000833801F50E944B2180FD88C063E58091EF
:101420000201909103010E941C220E945A132FEF87
:1014300081EE94E0215080409040E1F700C0000030
:1014400063E580910201909103010E941E22CF91D9
:101450000C945A138438C1F40E944B2182FD66C05B
:1014600067E480910201909103010E941C220E9476
:101470005A132FEF81EE94E0215080409040E1F725
:1014800000C0000067E4DDCF8CEF8C0F813AF8F4E8
:101490008C2F0E94F41F811149C06C2F8091020192
:1014A000909103010E94E621882349F06C2F8091DE
:1014B0000201909103010E941E220E945A136C2F78
:1014C00080910201909103010E941C22C0CF80E212
:1014D0008C0F883048F4C77081E001C0880FCA952E
:1014E000EAF70E941B13B3CFEBE5EC0FE33040F4B7
:1014F000F0E0E95BFE4F808190E0CF910C94AE214B
:10150000E8E5EC0FE73150F4F0E0EE0FFF1FE75E87
:10151000FE4F80819181CF910C94C421CD3E30F05B
:101520008C2F0E943E19CF910C94101ACF910895E0
:10153000882309F464C0823879F40E944B2181FF2A
:101540005EC069E380910201909103010E941C2218
:101550000E945A1369E310C08338B1F40E944B21F2
:1015600080FF4DC063E580910201909103010E94CC
:101570001C220E945A1363E580910201909103019D
:101580000E941E220C945A13843879F40E944B2135
:1015900082FF35C067E480910201909103010E94AF
:1015A0001C220E945A1367E4E7CF9CEF980F913AF0
:1015B00010F4682FE1CF90E2980F983050F48770C4
:1015C00091E001C0990F8A95EAF7892F0E942113B3
:1015D000D9CF9BE5980F933020F480E090E00C94F5
:1015E000AE2198E5980F973120F480E090E00C94BC
:1015F000C4218D3E20F00E9499190C94101A089570
:101600001F93CF93DF93182FEB010E94E9092097D6
:1016100041F08FE99FE00197F1F700C000002197AA
:10162000F6CF812FDF91CF911F910C94980A8933C7
:1016300019F060E070E002C060E570E00C94000B0F
:10164000882321F00E941B130C945A1308958823B9
:1016500021F00E9421130C945A130895CF92DF9227
:10166000EF92FF920F931F93CF93DF937C01D62FBE
:10167000C72FFC011281058102950F700E94111382
:101680008823B9F01123A9F08C2F807F803421F0BA
:1016900080E28D0F883068F08091880282FD09C059
:1016A00082E00E94BA130E94111391E0D82ED9262D
:1016B00001C0D12CCC2EC2948FE0C8228C2D90E09A
:1016C0008C30910508F0CFC1FC01EA5AFF4F0C9411
:1016D000D72A8C2F807FCF70882311F0C295C07FCE
:1016E000112399F0CC2309F4AAC180E28D0F883030
:1016F00010F0D11104C08C2F0E941B1303C08C2F3B
:101700000E942B130E945A139AC18D2F0E94980A8F
:10171000CC2309F4A8C180E28D0F883038F1DD2395
:1017200029F18C2F0E94311324C08C2F807FCF7021
:10173000803211F0C295C07FDD2319F0D130A1F1C4
:101740003DC08091880282FF17C0112349F0CC234D
:1017500029F08C2F0E941B130E945A1380E070C145
:1017600080E00E94980ACC2309F47DC18C2F0E944E
:1017700021130E945A1377C1112371F0002341F005
:10178000013031F40E943B138C2B0E9443136BC138
:101790000E943B138C2B1DC0002319F0013009F46B
:1017A00062C10E94501325C0112321F0063008F0B9
:1017B0005AC10EC0053008F056C11BC0112361F09C
:1017C000002331F0F701858180FF39C18F70858357
:1017D0008C2F0E94200B47C1002359F0D93309F008
:1017E0003FC1FFEF07EE13E0F15000401040E1F77A
:1017F00035C18C2F0E94270B36C18C2F869586957C
:10180000837019F0813061F02EC1112321F08D2FEA
:101810009C2F937002C080E090E00E94AE212BC10B
:10182000112321F08D2F9C2F937002C080E090E057
:101830000E94C42120C18D2F112319F00E943E194E
:1018400002C00E9499190E94101A15C18C2F837032
:1018500009F047C011110BC12D2F22952695277035
:10186000220F220F6D2F6F70862F90E0A0E0B0E066
:10187000022E04C0880F991FAA1FBB1F0A94D2F71B
:10188000D4FF10C04FE050E060E070E004C0440FAF
:10189000551F661F771F2A95D2F740955095609582
:1018A000709503C040E050E0BA01C695C695C3707C
:1018B0008A019B01082B192B2A2B3B2BC901B8014C
:1018C000C23049F058F4C13019F00E942F0ECFC039
:1018D0000E941D0ECCC00E94410EC9C00E941B0E6A
:1018E000C6C0112319F08C2F817001C08695882302
:1018F00009F4BDC02D2F229526952770220F220FA7
:101900006D2F6F70862F90E0A0E0B0E0022E04C033
:10191000880F991FAA1FBB1F0A94D2F7D4FF10C0CB
:101920004FE050E060E070E004C0440F551F661FB8
:10193000771F2A95D2F7409550956095709503C012
:1019400040E050E0BA01C695C695C3708A019B017C
:10195000082B192B2A2B3B2BC901B801C23049F0A7
:1019600058F4C13019F00E94F40E81C00E94E20EBA
:101970007EC00E94060F7BC00E94550E78C0CF70BB
:10198000112339F08C2F0E947B0E8D2F0E94200B8B
:101990006EC08D2F0E94270B8C2F0E949C0E67C05B
:1019A000D23F21F128F4D03F41F0D13FC1F043C0F4
:1019B000D33F19F1D43F79F03EC0112341F00530F7
:1019C00008F051C08C2F8F710E94C10E4CC00630A0
:1019D00008F049C0F7CF8091880282FF18C0112318
:1019E00039F08C2F8F710E947B0E3DC01123C9F3FB
:1019F0008C2F8F710E949C0E36C0112329F08C2FE2
:101A00008F710E94660E2FC00E94610E2CC01123A0
:101A100049F0CF718C2F0E947B0E63E08C2F0E94C7
:101A20009F1321C081E00E94BA130230E0F082E0EF
:101A30000E94BA1318C0112331F0002391F28D2FA8
:101A40000E94E90910C0002399F2D93349F41FEF2D
:101A500027EE33E0115020403040E1F700C0000095
:101A60008D2F0E94980A88EF8C0D843020F40E94FC
:101A70004B210E945709DD20C9F00E940D1380FD03
:101A800015C0F70112820E9407130E947B0EC70146
:101A90000E94770D0E940713DF91CF911F910F9144
:101AA000FF90EF90DF90CF900C949C0EDF91CF9140
:101AB0001F910F91FF90EF90DF90CF9008950F93BB
:101AC0001F93CF93DF93EC01688179818A810E9413
:101AD000BF0F8C010E94180F0E94090EB801CE01A1
:101AE0000E942E0BDF91CF911F910F910895CF93FC
:101AF000DF93EC01988189812B813C81232B31F08C
:101B00008F3F31F481E09F3F19F403C081E001C0B1
:101B100080E080FD1DC0CE010E94EE07811110C043
:101B20000E9411138823A1F08A81882389F0809173
:101B3000880282FD0DC082E0DF91CF910C94BA1330
:101B4000CE010E945F0DCE01DF91CF910C94CF07A3
:101B5000DF91CF91089580E090E00E94AE2180E077
:101B600090E00E94C4210E9438130E945A130E94E0
:101B7000C31B0C94101A80910201909103010E94E2
:101B800020220C94AB0D0E9428130C94BB0D92954F
:101B90009F70963079F010F4925001C09A509230B4
:101BA00068F4803F69F018F4883E40F409C0843F2F
:101BB00029F406C0883E20F0813F11F080E00895AE
:101BC00081E00895FC01808191810E94B40F0E9400
:101BD000C70D0895CF93DF9300D000D01F92CDB7EB
:101BE000DEB70F900F900F900F900F90DF91CF9175
:101BF0000895CF93DF9300D000D000D0CDB7DEB7EB
:101C000026960FB6F894DEBF0FBECDBFDF91CF9101
:101C10000895089508950C940A0E0C940B0E0E94DA
:101C20000D0E6093FB017093FC018093FD01909376
:101C3000FE010C94AB0D0C940F0E0F931F930091AB
:101C4000FB011091FC012091FD013091FE01602B00
:101C5000712B822B932B1F910F910C940F0E0F93CE
:101C60001F930091FB011091FC012091FD01309127
:101C7000FE0160237123822393231F910F910C9403
:101C80000F0E0F931F930091FB011091FC01209107
:101C9000FD013091FE0160277127822793271F9154
:101CA0000F910C940F0E0C940A0E0E94530E609329
:101CB000F7017093F8018093F9019093FA010C9465
:101CC000AB0D60E070E0CB010C94550E0F931F93A9
:101CD00041E050E060E070E08A019B0104C0000F29
:101CE000111F221F331F8A95D2F7C901B8011F9116
:101CF0000F910C94550E0F931F9341E050E060E05C
:101D000070E004C0440F551F661F771F8A95D2F7F5
:101D10008091F7019091F801A091F901B091FA0139
:101D20008A019B01082B192B2A2B3B2BC901B801D7
:101D30001F910F910C94550E0F931F9341E050E0AB
:101D400060E070E004C0440F551F661F771F8A953E
:101D5000D2F740955095609570958091F7019091DC
:101D6000F801A091F901B091FA018A019B010823C1
:101D700019232A233B23C901B8011F910F910C9409
:101D8000550E0F931F9341E050E060E070E004C0F7
:101D9000440F551F661F771F8A95D2F78091F70170
:101DA0009091F801A091F901B091FA018A019B018B
:101DB000082719272A273B27C901B8011F910F912E
:101DC0000C94550E0F931F930091F7011091F80199
:101DD0002091F9013091FA01602B712B822B932B0A
:101DE0001F910F910C94550E0F931F930091F701C3
:101DF0001091F8012091F9013091FA0160237123CB
:101E0000822393231F910F910C94550E0F931F93D0
:101E10000091F7011091F8012091F9013091FA0138
:101E200060277127822793271F910F910C94550EDD
:101E30000895292F220F920F990F890FE82FE69509
:101E4000E695E695877051E001C0550F8A95EAF74F
:101E500085E0E89FF0011124EE50FE4F20E030E0D5
:101E600070E04081CB01022E02C0969587950A94BE
:101E7000E2F78170819584278523842781932F5FE2
:101E80003F4F2530310569F70895292F220F920F12
:101E9000990F890F682F669566956695982F9770AC
:101EA00085E0689FB001112440E050E080E0FB0134
:101EB000E40FF51FEE50FE4F208130E0092E02C0E6
:101EC000369527950A94E2F721703327042E01C036
:101ED000220F0A94EAF7822B4F5F5F4F453051057E
:101EE00031F70895BF92CF92DF92EF92FF920F9356
:101EF0001F93CF93DF938C01C090F701D090F8012E
:101F0000E090F901F090FA018091FB019091FC01C1
:101F1000A091FD01B091FE01C82AD92AEA2AFB2A24
:101F2000CFE1D0E0D701C6010C2E04C0B695A7952D
:101F3000979587950A94D2F780FD04C0219790F772
:101F4000B12C07C0BC2EB8018C2F0E949A160197A5
:101F5000A9F38B2DDF91CF911F910F91FF90EF90FF
:101F6000DF90CF90BF900895CF93DF93EC010E9454
:101F7000720FBE010E949A16DF91CF9108951F93B0
:101F8000CF93DF93EB019091F101992321F0CB01E5
:101F90000E94B40F13C0882349F0CB010E94720F36
:101FA000182F682FCE010E94190F04C0CB010E9488
:101FB000450F182FBE01812F0E949A16DF91CF91F5
:101FC0001F9108951F93CF93DF93C091FF0116E0F7
:101FD00080910002C81799F0D0E01C9FF0011D9F6E
:101FE000F00D1124EF5FFD4F4081518162817381BB
:101FF000848195810E94F90D2196C770E9CFDF9108
:10200000CF911F9108954091310250913202609119
:1020100033027091340280913502909136020C9413
:10202000F90DEF92FF920F931F93CF93DF9380915F
:10203000360282958F7009F065C080913302882343
:1020400009F460C08091FF01F0900002109131020C
:1020500000913202609134027091350291E01F3F8D
:1020600009F090E0C0910001D0910101292F96E084
:10207000E92E8F1509F446C06115710521F00F3F57
:1020800021F030E003C031E001C0322F90E030FD9C
:1020900036C0E89EF001E99EF00D1124DF01AF5F2C
:1020A000BD4F11963C911197301329C03C913113CB
:1020B00026C012963C911297311121C013964D9172
:1020C0005C911497461B570B4C175D07C0F4809129
:1020D00036028F70806180933602EA5FFD4F808107
:1020E0008F708061808381E392E00E94770DDF91A1
:1020F000CF911F910F91FF90EF900C94E20F0196FA
:102100008770B7CFDF91CF911F910F91FF90EF9024
:1021100008959F92AF92BF92CF92DF92EF92FF927B
:102120000F931F93CF93DF93CDB7DEB761970FB6B1
:10213000F894DEBF0FBECDBF8C0185E0F801DE0153
:102140001D9601900D928A95E1F7D8011296EC90B8
:1021500090913102E09132022091340230913502A7
:102160002115310531F0EF3F31F481E09F3F19F443
:1021700003C081E001C080E0B82FB1709B2E80FDCC
:1021800047C1D8014C9111965C9111971396AD906F
:10219000BC90149781E3C82E82E0D82EF0903302D1
:1021A000B501621B730B2091000130910101FF20EA
:1021B00009F4D9C0809136026217730708F095C000
:1021C000282F207F09F052C05E1313C0491311C09D
:1021D000FE2CE1100EC08F708061809336020E9449
:1021E0000310C6010E94770D80913602F8018583A5
:1021F0004DC1AB2831F05F3F31F481E04F3F19F41E
:1022000003C081E001C080E080FD03C081E08E2535
:1022100002C080E090E0F82FF170FF2E80FF1CC01C
:102220008091FF012091000236E0821709F40BC172
:1022300090E0389FF001399FF00D1124EF5FFD4FC2
:102240006181561306C06081461303C06281E612A5
:1022500003C001968770E9CFFE2CEE2009F416C169
:102260008091360281608093360254C05E1306C0AE
:10227000491304C0E11002C0F80199C0C8010E94CE
:10228000E20D882361F1EE2051F120913602822F78
:1022900082958F7090E0029774F080913102909156
:1022A000320298878F831986BB86AA862C87CE0137
:1022B00007960E94770D86E0F801A1E3B2E0019055
:1022C0000D928A95E1F70E9411100E9403100AC036
:1022D0005E1711F1C8010E94E20D81112CC0C801E6
:1022E0000E94770DFF24F394D1C0282F207F81F71F
:1022F0007A2DB98AA88A6E2D89890E94EA0D81E318
:1023000092E00E94770D86E0D6011D928A95E9F74A
:102310000E940310F12CBAC04913DCCFE110DACFD0
:10232000F8018583C8010E94770D86E0D6011D92D1
:102330008A95E9F7ABC0EE2091F220913602822F08
:1023400082958F7090E002970CF4B5CF80913102A6
:10235000909132029A8389831B82BD82AC822E8344
:10236000CE010196A6CF6217730708F044C0FE2C79
:10237000EE2009F4B4CF5E1330C049132EC0209173
:10238000360220FD21C0822F82958F70482F50E0A9
:1023900041155105C9F0F80125834F30510541F031
:1023A0008F5F982F9295907F822F8F70892B8583D6
:1023B000C8010E94770D86E0F801A1E3B2E0019028
:1023C0000D928A95E1F73CC086E0F801A1E3B2E006
:1023D00001900D928A95E1F759C0C8010E94E20D63
:1023E000811169CF80913602816080933602C801E5
:1023F0000E94770D4BC07A2DB98AA88A6E2D8989E3
:102400000E94EA0D86E0D6011D928A95E9F718C070
:10241000EE2009F464CFC8010E94E20DF82E882353
:1024200009F45DCF86E0F801A1E3B2E001900D92DE
:102430008A95E1F781E392E00E94E3090E9411107E
:102440000E94031023C04D875E878D859E850E9464
:10245000B40F292F22952F70223028F49F7039F065
:10246000811105C00BC0243028F49F7049F4805EB0
:10247000883020F0C8010E94770D9F2CF92C06C0EF
:10248000D80115969C91907F91F7F8CF8F2D61968A
:102490000FB6F894DEBF0FBECDBFDF91CF911F9175
:1024A0000F91FF90EF90DF90CF90BF90AF909F90F3
:1024B00008951F93CF93DF93CDB7DEB72C970FB658
:1024C000F894DEBF0FBECDBF4F83588769877A87E8
:1024D0008B879C87CE0107960E9489108823D1F0B4
:1024E0009F8188852A853B85232B31F08F3F31F4EE
:1024F00081E09F3F19F403C081E001C080E080FDCE
:1025000047C04F81588569857A858B859C850E9457
:10251000F90D3EC086E0FE013796DE01119601906E
:102520000D928A95E1F7FF81E8856A857B856115C3
:10253000710531F0EF3F31F481E0FF3F19F403C042
:1025400081E001C080E080FD23C02091000230E0E6
:10255000C9010196877099274091FF0150E08417C7
:102560009507F1F1F983EA837D836C8396E0929F6E
:10257000D001939FB00D1124AF5FBD4FFE01319686
:1025800001900D929A95E1F7809300020E94E20F6C
:1025900016E08091FF0190910002891771F1189F58
:1025A000C00111248F5F9D4F0E948910882329F15B
:1025B000E091FF011E9FF0011124EF5FFD4F40816C
:1025C000518162817381848195810E94F90D80918E
:1025D000FF0190E00196877099278093FF01D9CF82
:1025E0000E94C30D109200021092FF01E1E3F2E09D
:1025F00086E0DF011D928A95E9F72C960FB6F894D4
:10260000DEBF0FBECDBFDF91CF911F9108958091A6
:102610003F02859585958595089580913F02877045
:10262000089590913F02977081E009F480E0089549
:1026300080914A02089590914A02892B80934A0220
:102640000895809590914A02892380934A020895C3
:1026500010924A02089590914902892B8093490271
:1026600008958095909149028923809349020895A5
:1026700010924902089580914002089508950C94A3
:102680003E130C943F139091880292FD08C09091E4
:102690004002981721F0809340020C944113089552
:1026A00080914002882329F01092400280E00C942F
:1026B00041130895CF93DF93E0910201F09103015C
:1026C00080914A028083E0910201F09103019081A0
:1026D00080914902892B808380914002882381F078
:1026E000E0910201F09103019081892B8083809118
:1026F0000201909103010E94DA2181110E9450137E
:10270000C0910201D091030148E050E067E372E01C
:10271000CE010E94F12A892B69F088E0FE01A7E32F
:10272000B2E001900D928A95E1F7CE01DF91CF9151
:102730000C945721DF91CF9108950C943E13909102
:10274000880292FD10C098E0899F90011124262BE9
:1027500020933F020E947B0E80913F0285958595D4
:1027600085950C949D130C947B0E10923F0280E093
:102770000C949D1320913F028095822380933F0209
:10278000982F977099F430E0482F082E000C550BC5
:102790002417350759F09091880292FD07C085955E
:1027A000859585950E949C0E0C94B5130895CF9342
:1027B0009091880292FB222720F92817F9F0C82F60
:1027C000892FC0FB82F980938802809187029091C3
:1027D00088020E94331482E00E94BA13809154024E
:1027E00080FF0CC01F92CF9387E892E09F938F9356
:1027F0000E947A060F900F900F900F90CF9108953E
:102800008091880282FB882780F991E089270C94C7
:10281000D71381E00C94D71380E00C94D71380E099
:1028200090E00E94062B21E0893E9E4F09F020E0B7
:10283000822F089582E090E00C94FE2A83E090E0DD
:102840000C94FE2ACF9384E090E00E94FE2AC82FC9
:1028500082E290E00E94FE2A2C2F30E0A901582B42
:10286000CA01CF910895CF93C92F682F84E090E0DB
:102870000E940C2B6C2F82E290E0CF910C940C2BD9
:10288000AB01BC018FE090E00C941E2BAB01BC01AE
:1028900083E190E00C941E2B60E070E0CB010C947F
:1028A000461460E070E0CB010E9440140C944C147C
:1028B00069EE7EEF80E090E00E942A2B60E082E0EB
:1028C00090E00E940C2B60E083E090E00E940C2BD3
:1028D0001092FB011092FC011092FD011092FE017A
:1028E00060E084E090E00E940C2B60E082E290E0E7
:1028F0000E940C2B60E085E090E00E940C2B60E0D1
:1029000086E090E00E940C2B6FEF87E090E00E9441
:102910000C2B40E050E0BA0188E090E00E941E2BB2
:1029200060E08DE090E00E940C2B40E050E0BA01A6
:1029300088E190E00E941E2B60E087E190E00E9419
:102940000C2B40E050E0BA018CE190E00E941E2B7D
:1029500060E070E080E290E00E942A2B40E050E0CE
:10296000BA0188E190E00E941E2B0C9451140C9443
:102970005814682F8EE090E00C940C2B0E94C92212
:1029800060935002709351028093520290935302CD
:1029900060934C0270934D0280934E0290934F02CD
:1029A000089585B7806885BF85B7806885BF08951D
:1029B00081E008950C94D81408950C94DC140C94C0
:1029C000DC140C94DF140C94DC140C94E3140C94BD
:1029D000DC140E94D11481E095E20E9441210E9402
:1029E000E7140C94E5140E94DD140C94DC140E948E
:1029F00077170C9456090E94B4220E9445180E9431
:102A0000F7140C94E114DF92EF92FF920F931F934F
:102A1000CF93DF93CDB7DEB72A970FB6F894DEBF1A
:102A20000FBECDBF0E945018D82E81110E94BE1437
:102A300080E00E949B17F82EE0904B02E82689F474
:102A40008FEF89838A831B820E94BD228160782F49
:102A50009D838C8349815A816B818D810E94990964
:102A60002CC08091540281FD0E94A11700E011E06A
:102A70008E2D8123E9F00E94DA14882399F00E83C9
:102A80001F82F12281E009F480E088870E94BD2244
:102A90008160782F9A8789874E815F8168858A85D2
:102AA0000E94990980914B02182710934B0205C090
:102AB0000F5F110F0630E1F6C3CF81E0D11001C0E6
:102AC00080E02A960FB6F894DEBF0FBECDBFDF912F
:102AD000CF911F910F91FF90EF90DF9008950E948A
:102AE00003150E94B01A0C946709CF93DF930E94DC
:102AF0009F16EC01811521E5920708F045C081156C
:102B000030E5930708F094C0883E910528F5803E93
:102B1000910508F0F8C0883A910570F4853A91055E
:102B200008F07CC08130910509F475C008F4E8C054
:102B3000049708F0E8C0E4C08F3B910508F0E0C0BE
:102B4000C85AD0E0CC0FDD1FC65BDE4F0990D8819C
:102B5000C02DCE019464D8C0811540E2940758F48A
:102B6000811551E0950708F0CEC08D3E910508F41F
:102B7000C7C09065C9C0C11580E4D80708F4C0C0BB
:102B8000DF70CE01906AC0C0811525E59207A8F4D8
:102B9000811534E5930708F095C0811543E5940746
:102BA00008F07BC0811552E5950708F061C0D82F69
:102BB000CC27CE01816F906AA7C0C11589E5D807DF
:102BC000A0F4C11528E5D20708F082C0C11536E58A
:102BD000D30708F095C08C2F0E9433178F7190E0B7
:102BE000D82FCC27CE0190628FC0C1154AE5D407FB
:102BF00008F474C0CE0190568115904208F080C050
:102C00008D2F8F710E943317DD27D0628F71AE0137
:102C1000582BCA0179C081E090E076C0C55AD0E057
:102C2000C858DE4F8881C82FD0E0CE0190646CC0B8
:102C300074E0969587957A95E1F7282F23703C2FBD
:102C4000337081E090E002C0880F991F3A95E2F757
:102C50009C68AC01522B9A019C2F9F70969596957B
:102C600050E2959FE0011124C9018C2B9D2B4CC093
:102C70008370992721E030E002C0220F331F8A952C
:102C8000E2F79C2F9695969580E2989FE00111249B
:102C9000C22BD32BCE019C6837C08370992721E0CB
:102CA00030E002C0220F331F8A95E2F79C2F9695E1
:102CB000969540E2949FE0011124C22BD32BCE01C4
:102CC0009A6822C0D82FCC27CE01846F906A1CC08E
:102CD000DC2FCC27CE01806F906A16C08C2F8F70AE
:102CE0000E94331794E0D695C7959A95E1F7CF7077
:102CF000D0E0DC2FCC27D0699E01282BC90104C06D
:102D000080E090E001C0CE01DF91CF910895272FA0
:102D100030E0280F311D86E0829FF001839FF00D87
:102D20001124E60FF11DEE0FFF1FEE51FF4F8591AD
:102D3000949108950E9487160E947515089582380F
:102D4000910569F1B0F48133910509F46DC048F43F
:102D50008932910509F463C08A32910509F469C08A
:102D600008958533910509F455C089339105B9F06B
:102D70000895833E910569F138F4803E9105B1F0E4
:102D8000823E910509F10895863E9105A9F1873E9D
:102D90009105B9F1843E910509F064C023C02091EA
:102DA000870220FD4FC021FD4DC00895809187020C
:102DB00080FD44C08091880280FF44C080918702DA
:102DC00084FD42C083EE4DC08091870282FF38C0EF
:102DD000F5CF8091870282FD33C08091880280FD0B
:102DE00031C0ECCF8091880281FF32C08091870290
:102DF00084FD2AC087EE35C08091870283FF26C0FC
:102E0000F5CF8091870283FD21C08091880281FDEA
:102E10001FC0ECCF8091870285FD1CC01DC0809132
:102E2000870285FD19C016C08091870286FD16C0F5
:102E300017C08091870286FD13C010C089E311C0BE
:102E400082EE0FC080EE0DC080E00BC086EE09C0A0
:102E500084EE07C089E205C085E303C08AE201C0B1
:102E600081E390E008959091870292FF0DC0282F92
:102E70002871283019F4877F846006C0282F2471B8
:102E8000243011F48B7F886093FF0DC0282F2871A8
:102E9000283119F4877E846106C0282F24712431DB
:102EA00011F48B7E88612091880220FF0DC0382F9D
:102EB0003871383019F4877F816006C0382F31713E
:102EC000313011F48E7F886021FF0DC0282F2871CA
:102ED000283119F4877E816106C0282F21712131A4
:102EE00011F48E7E886194FD877E089508950E9476
:102EF0000F14811102C00E94B7140E941A1480930B
:102F000054020E94221490938802809387020E94A8
:102F100076170E941E14682F70E080E090E00E94F7
:102F20001B0E6091F7017091F8018091F901909169
:102F3000FA010C94530EE82FF0E0E657FD4F808124
:102F400008958BEA92E00E94E1051F921F9286EAA3
:102F500092E09F938F930E947A0683EA92E00E9408
:102F6000E10580918A020E943D091F928F938EE9AC
:102F700092E09F938F930E947A068DB79EB7089632
:102F80000FB6F8949EBF0FBE8DBF8CE992E00C94F3
:102F9000E10580EA8A95F1F7089500C008950C9440
:102FA000C91708950C94D1170C94D2170C94EA0603
:102FB000F894E82FE295EF70F0E031A1282F2F7000
:102FC00081E090E001C0880F2A95EAF7982F90954C
:102FD000932391A392A1892B82A3789408950F93B0
:102FE0001F93CF93DF9380E90E94D817CBE7D1E0FE
:102FF00001E811E089918F3F11F00E94D8170C175A
:103000001D07C1F7DF91CF911F910F9108950F9385
:103010001F93CF93DF938C01D62FF894509A589832
:1030200078940E94CD17EBE7F1E031E0C0E0219108
:103030002F3F89F0A22FA295AF70B0E090968C91AF
:1030400090E02F7002C0959587952A95E2F780FD54
:1030500002C0832F01C080E0C82B330F81E0E1382C
:10306000F80729F780E90E94D81761E0C11101C073
:1030700060E08D2F0E94CF17F801ED0FF11DC08386
:10308000DF91CF911F910F9108950E94EF17109239
:103090008A021092890281E00E9476180C94DA0765
:1030A0001F93CF93DF931F92CDB7DEB7198260E0F5
:1030B000CE0101960E94071890918902898111E042
:1030C000981301C010E0981380938902212F41E0EA
:1030D0006AE872E089E892E00E9477180E94DC07B3
:1030E000812F0F90DF91CF911F9108950895FF9246
:1030F0000F931F93CF93DF938C01F62ED72FC42FFE
:10310000222349F081E0809357020E94BD229093D0
:10311000560280935502809157028823C1F0809116
:103120005502909156020E94D522059780F0EF2D0E
:10313000FD2FD8014C2F50E0CD01801B910B84173F
:1031400095071CF48D918193F7CF10925702DF9170
:10315000CF911F910F91FF9008950E947D250E94AD
:10316000FB140C9489250E948D250E946F150C94E8
:10317000AB250E945B220E9464250E94E9140E94F4
:10318000AD180E94B3180E94F314FBCF80915E0229
:1031900080FF06C06091090170E0660F771F26C0AE
:1031A00081FF04C06091090184E005C082FF07C06F
:1031B0006091090188E0689FB001112417C09091C7
:1031C0005D029923D1F060910801961788F720914C
:1031D000090188E0289F90011124929FA001939FEC
:1031E000500D112470E0CA010E94C32A6038710595
:1031F00040F46115710519F406C068E070E0862F8F
:1032000008958FE7089581E0089580915E0280FF20
:1032100008C06091050170E0759567957595679593
:1032200021C081FF06C06091050170E0759567952A
:1032300019C082FF04C06091050170E010C0909138
:103240005C02992399F0609104019617A0F7809190
:103250000501899FC001112470E00E94C32A6038D3
:10326000710540F46115710519F406C061E070E064
:10327000862F08958FE7089581E008958D3E21F40B
:103280000E94C618819504C08E3E29F40E94C6187B
:103290008093620208958F3E21F40E94C6188195A2
:1032A00004C0803F29F40E94C618809361020895EB
:1032B000893F19F40E94051905C08A3F31F40E9424
:1032C000051981958093630208958B3F21F40E9434
:1032D0000519819504C08C3F29F40E94051980933B
:1032E000640208959FE0980F983078F421E030E070
:1032F000A90102C0440F551F9A95E2F7CA019091A7
:103300006002892B8093600208958D3F21F48091A3
:103310005E0281600BC08E3F21F480915E0282606C
:1033200005C08F3F29F480915E02846080935E0225
:1033300008958D3E39F49091620297FF35C0109246
:10334000620259C08E3E29F4909162021916BCF3B4
:103350002BC0909161028F3E29F497FF25C01092F7
:10336000610249C0803F19F41916CCF31DC0909139
:103370006302893F29F41916BCF4109263023BC022
:103380008A3F19F497FF10C0F8CF8B3F39F4909122
:10339000640297FF09C0109264022DC08C3F21F493
:1033A000909164021916BCF39FE0980F983080F456
:1033B00021E030E0A90102C0440F551F9A95E2F7C1
:1033C000CA0180959091600289238093600213C0A6
:1033D0008D3F21F480915E028E7F0BC08E3F21F4E1
:1033E00080915E028D7F05C08F3F29F480915E023F
:1033F0008B7F80935E0280916102811106C0809173
:103400006202811102C010925D02809163028111FB
:1034100006C080916402811102C010925C0208957E
:103420008091540283FF7EC081EE92E00E94E1050C
:10343000809160021F928F938CED92E09F938F9307
:103440000E947A068AED92E00E94E1058091610275
:10345000282F082E000C330B3F938F9387ED92E0BB
:103460009F938F930E947A0685ED92E00E94E1057A
:1034700080916202282F082E000C330B3F938F930C
:1034800082ED92E09F938F930E947A0680ED92E006
:103490000E94E10580916302282F082E000C330B57
:1034A0003F938F938DEC92E09F938F930E947A06C7
:1034B0008BEC92E00E94E10580916402282F082E97
:1034C000000C330B3F938F9388EC92E09F938F9384
:1034D0000E947A0685EC92E00E94E10580915D02EF
:1034E0001F928F9382EC92E09F938F930E947A06B3
:1034F00080EC92E00E94E10580915E021F928F9322
:103500008DEB92E09F938F930E947A068AEB92E074
:103510000E94E1058DB79EB74C960FB6F8949EBFFA
:103520000FBE8DBF0E94BD2220916102211104C0F7
:1035300020916202222321F090935B0280935A0231
:1035400020916302211104C020916402222321F002
:1035500090935902809358028FE592E00C94A02139
:10356000EF92FF920F931F93CF93DF9300D000D081
:1035700000D0CDB7DEB786E0EFE5F2E0DE011196D0
:1035800001900D928A95E1F7E0906102F09062025D
:103590000091630210916402109261021092620223
:1035A0001092630210926402E11003C0FF2009F43C
:1035B0005DC080915A0290915B020E94D522AC01BD
:1035C00090915D02992339F020910A0130E024178F
:1035D000350758F04BC020910B018AE0289F9001DD
:1035E00011242417350718F041C09F3F19F09F5F41
:1035F00090935D02EE2061F00E94C6181E1414F034
:103600009FEF01C091E0989F902D1124909361024B
:10361000FF2061F00E94C6181F1414F09FEF01C034
:1036200091E0989F902D1124909362023091610255
:103630003323E1F0209162022223C1F045EB3403F1
:10364000C0011124992319F09093610203C081E015
:103650008093610235EB2303C0011124992319F0F3
:103660009093620203C081E080936202011103C063
:10367000112309F45DC080915802909159020E9473
:10368000D522AC0190915C02992339F0209106017A
:1036900030E02417350758F04BC0209107018AE02D
:1036A000289F900111242417350718F041C09F3F2F
:1036B00019F09F5F90935C02002361F00E9405194E
:1036C000101614F09FEF01C091E0989F902D1124E7
:1036D00090936302112361F00E940519111614F0F2
:1036E0009FEF01C091E0989F902D11249093640268
:1036F000309163023323E1F0209164022223C1F070
:1037000045EB3403C0011124992319F0909363020F
:1037100003C081E08093630235EB2303C0011124D1
:10372000992319F09093640203C081E080936402AE
:103730008091610281110BC080916202811107C0EA
:1037400080916302811103C08091640281110E9403
:10375000101AEB82FC820D831E8386E0FE013196F7
:10376000AFE5B2E001900D928A95E1F726960FB68B
:10377000F894DEBF0FBECDBFDF91CF911F910F91A7
:10378000FF90EF900895EFE5F2E086E0DF011D92F3
:103790008A95E9F710925D0210925C0210925E0227
:1037A0000895CF93DF93EC01FB018281882309F414
:1037B0003CC1C430FDE5DF0760F4CB3F9CE5D90791
:1037C00088F49E0122503C452431310508F02EC179
:1037D00009C0C236EDE5DE0729F0C63AFDE5DF0790
:1037E00009F024C10E9422149093880280938702DA
:1037F000C1318CE5D80709F4C6C008F042C0C93011
:10380000ECE5DE0709F49BC000F5C5308CE5D80770
:1038100009F485C078F4C330ECE5DE0709F478C01C
:1038200008F07AC0C230DC4509F0F5C0809187020B
:103830008160EFC0C7309CE5D90709F478C008F073
:103840007AC0809187028061E4C0CD30FCE5DF075B
:1038500009F487C058F4CB309CE5D90709F479C046
:1038600008F07BC08091870288606FC0CF30FCE594
:10387000DF0709F480C008F082C080918702877F4B
:10388000C8C0CE3F9CE5D90709F471C000F5C53129
:10389000FCE5DF0709F485C068F4C3319CE5D9076E
:1038A00009F475C008F095C00E94C30D809187028D
:1038B0008F77AFC0CC3FFCE5DF07A9F108F054C01B
:1038C000CB3FDC4509F0A7C08091880240C0C230E0
:1038D000EDE5DE0709F489C058F4C1158DE5D80778
:1038E00009F45AC008F069C08091880282602FC034
:1038F000C236EDE5DE0709F47CC0C63AFDE5DF0718
:1039000009F481C0C330DD4509F085C080E06EC098
:103910008091870282607DC08091870216C080916D
:103920008702886076C08091880282604FC0809153
:10393000870280626EC08091870280646AC00E94A4
:10394000C30D80918702806864C0846062C081601A
:103950003DC0809187028E7F5CC0809187028D7F01
:1039600058C08091870216C08091880218C080914B
:1039700088028D7F2BC0809187028F7E4AC0809104
:1039800087028F7D46C0809187028F7B42C08091E5
:103990008702877F8B7F3DC0809188028D7F8E7FDD
:1039A00015C08091870282FB222720F991E092279F
:1039B00090FB82F990FB83F92CC080918802982FAC
:1039C000909591708E7F892B90FB81F9809388026E
:1039D00022C00E94C30D8091870287FB222720F915
:1039E00091E0922790FB87F914C081E00E94B914FE
:1039F00012C08091870284FB222720F991E0922750
:103A000090FB84F906C080918702982F909590FBD7
:103A100080F98093870280918702909188020E94AA
:103A200033140E94C30D80E001C081E0DF91CF918B
:103A30000895809104011F928F93809105011F9238
:103A40008F93809108011F928F93809109011F929B
:103A50008F9380910A011F928F9380910B011F9287
:103A60008F9384E093E09F938F930E947A068DB7A3
:103A70009EB70E960FB6F8949EBF0FBE8DBF0895E9
:103A8000883220F58E3108F068C08B3091F1C0F497
:103A9000873009F0BEC081E080930B0184E1809300
:103AA0000A018AE0809309018EE18093080188E091
:103AB0008093050188E28093040186E694E0C6C005
:103AC000833109F443C0843169F1A3C08F3409F410
:103AD0009EC028F4893231F1883359F09AC081357B
:103AE00031F008F4D4C0823509F4A7C092C08FEF3A
:103AF000A5C088E894E00E94E1050E94191D1F926C
:103B000081E08F931F9288E08F9381E893E09F93E9
:103B10008F930E947A060F900F900F900F900F9046
:103B20000F9096C085E894E00E94E10580916902BB
:103B3000882309F4AAC010926902109268021092B8
:103B400067021092660210926502B1C087E794E0A6
:103B50000E94E1050E94191D7BC08D51809369026E
:103B6000833031F170F48130D1F0823009F03FC000
:103B70008AE091E090936802809367028EE891E07A
:103B80001FC0853059F108F1863089F584E091E055
:103B9000909368028093670289EC91E011C08BE0FA
:103BA00091E0909368028093670285E891E008C0F5
:103BB00089E091E090936802809367028AE991E03E
:103BC000909366028093650218C088E091E090931C
:103BD00068028093670287EA91E0F2CF85E091E086
:103BE000909368028093670286EB91E0E9CF109290
:103BF000690284E794E00E94E105809169028823CC
:103C000009F455C01F928F9380E794E00DC08AE0BD
:103C100015C083E694E01AC097FF47C010828081E8
:103C20001F928F938DE594E09F938F930E947A0665
:103C30000F900F900F900F900BC081E0E091670202
:103C4000F0916802309729F58AE594E00E94E10539
:103C500020916902222359F18091650290916602B8
:103C6000009711F481E891E09F938F931F922F9317
:103C700081E594E09F938F930E947A060F900F90B6
:103C80000F900F900F900F9016C080E0089586EF70
:103C9000D5CF2081082E000C990B820F911D8F3FEC
:103CA000910509F00CF4B8CF8FEF8083B8CF8DE485
:103CB00094E00E94E10581E00895CF93C82F1F9200
:103CC0008F938EE994E09F938F930E947A0681E010
:103CD00090E0A0E0B0E0BC01CD0104C0660F771F0A
:103CE000881F991FCA95D2F70E941B0E0F900F9044
:103CF0000F900F90CF910C94C30DEF92FF920F9302
:103D00001F93CF93DF938B3109F4EDC008F08EC081
:103D10008B3009F4B1C008F078C0863009F4AFC028
:103D200020F4853009F4BDC04EC1873009F4C0C00D
:103D3000883009F048C10E941E141F928F9387ECAF
:103D400098E09F938F930E947A060E941A1483FB37
:103D5000992790F91F929F9382FB992790F91F92C0
:103D60009F9381FB992790F91F929F93982F9170B1
:103D70001F929F931F928F938EE798E09F938F934C
:103D80000E947A060E94221487FB222720F91F92A4
:103D90002F9386FB222720F91F922F9385FB222742
:103DA00020F91F922F9384FB222720F91F922F9333
:103DB00083FB222720F91F922F9382FB222720F9D1
:103DC0001F922F9391FB222720F91F922F93292FC7
:103DD00021701F922F9381FB222720F91F922F938E
:103DE000282F21701F922F939F938F9389E997E03B
:103DF0009F938F930E947A068DB79EB788960FB6D1
:103E0000F8949EBF0FBE8DBF35C0803109F495C0B8
:103E100020F48E3009F47BC0D6C0863109F4A8C0E6
:103E2000893109F0D0C08EE095E084C08A32E1F09B
:103E300060F4873209F4C3C028F48E3108F4C3C09B
:103E40008D51BEC0893269F1BEC0833448F48A33D3
:103E500008F0B3C0853309F4B2C0883369F0B3C049
:103E6000833409F4ACC0AFC082E799E00E94E10559
:103E70000E94B714C1E0ACC086EF95E05BC08091B2
:103E80005402817F8E7F809354028FEC95E00E94D4
:103E9000E1058EE699E00E94E10581E080936A02E7
:103EA000E9CF82E599E00E94E1050E94DF07E2CFB9
:103EB00080915402C82FC095C170C0FB80F98093D7
:103EC0005402CC2329F086E499E00E94E10580C0E9
:103ED00089E399E00E94E10580915402897F877F00
:103EE00080935402C7CF9091540291FBCC27C0F924
:103EF00081E0C827892FC0FB81F980935402CC232D
:103F000019F08CE299E029C08EE199E013C09091FC
:103F1000540292FBCC27C0F981E0C827892FC0FB4F
:103F200082F980935402CC2319F08FE099E015C0F8
:103F30008FEF98E00E94E1059DCF9091540293FB92
:103F4000CC27C0F981E0C827892FC0FB83F9809373
:103F50005402CC2351F083EF98E00E94E105809158
:103F6000540281608093540233C086EE98E0E2CF21
:103F70000E94C922162F072FF82EE92ED091860213
:103F8000C09118010E944B21EF92FF920F931F9353
:103F90001F92DF931F92CF931F928F9383EA94E037
:103FA0009F938F930E947A068DB79EB70C960FB69B
:103FB000F8949EBF0FBE8DBF5DCF895301C080E0D6
:103FC0000E945D1E57CF84EE98E00E94E105C0E09C
:103FD0008C2FDF91CF911F910F91FF90EF9008955B
:103FE00080E008950C94F01FCF93C82F80916A024F
:103FF000813071F040F0823009F045C08C2F0E9472
:10400000401D81E046C00E9418138232F1F504C0C1
:104010000E941813823261F48C2F0E94F21F8111CA
:1040200004C08C2F0E947D1E2CC081E090E029C02E
:104030008C2F0E94F01F811123C0C431C9F058F4A5
:10404000CB3069F0C031B9F482E080936A0288E332
:104050000E94401D15C0C93259F0C83361F48FEC7D
:1040600095E00E94E1058AE994E00E94E10508C01C
:1040700010926A020CC088E994E00E94E10507C032
:1040800081E0817006C010926A0280E002C080E088
:10409000F8CFCF910895CF93DF9386319C4541F5BA
:1040A000EB010E941813982F8A8120910201309110
:1040B0000301882379F09A7A81E009F480E0809303
:1040C0006B02911102C069E201C065E3C9010E945F
:1040D0001C220AC080916B02811102C069E201C0FA
:1040E00065E3C9010E941E220E945A1380E001C0AC
:1040F00081E0DF91CF9108950F931F93CF93DF93CA
:10410000C42FD22FFC0182818823C9F040936E0214
:104110000E94BD2290936D0280936C0280E28C0F0E
:10412000883008F057C0C77081E001C0880FCA9579
:10413000EAF7DF91CF911F910F910C94200B8091A2
:104140006E02481330C080916C0290916D020E9403
:10415000D522883C910538F510E21D0FCD17B9F036
:1041600080E28C0F883040F4C77081E001C0880F76
:10417000CA95EAF70E94270B183028F581E09D2F99
:10418000977001C0880F9A95EAF70E94200B802F44
:104190000E94170B1830F0F4D77081E001C0880F2F
:1041A000DA95EAF70AC080E28C0F883098F4C7707D
:1041B00081E001C0880FCA95EAF7DF91CF911F9186
:1041C0000F910C94270B802FDF91CF911F910F91AE
:1041D0000C94170BDF91CF911F910F9108950F93BE
:1041E0009C01CB01243F4CE5340731F188F4293D93
:1041F000FCE53F07D9F02A3D4CE5340779F1283D2D
:104200003C45A9F506E221EE41EE68ED7CE52BC0C8
:10421000263FFCE53F07E1F0A8F0273F3C4539F594
:1042200007E225EE46EE67EF7CE51DC007E225EECE
:1042300045EE69ED7CE517C006E221EE40EE64EF45
:104240007CE511C007E225EE44EE65EF7CE50BC08E
:1042500006E221EE42EE66EF7CE505C008E221E0D1
:1042600045EE6AED7CE50E947C2080E008C0FC0100
:104270008281882319F010926E0201C081E00F91B3
:1042800008959093EF018093EE0108959093740246
:10429000809373020895E0917302F0917402309755
:1042A00021F00190F081E02D099480E00895EF92D3
:1042B000FF920F931F93CF93DF93E0917302F091DE
:1042C00074023097B1F18C010280F381E02D0995E1
:1042D0008091540282FF2DC080FF04C08BE899E0DA
:1042E0000E94E105E80118E085E8E82E89E0F82E53
:1042F0008091540280FF0BC088811F928F93FF92A0
:10430000EF920E947A060F900F900F900F9011502D
:1043100021961111EDCF8091540280FF0AC083E8ED
:1043200099E0DF91CF911F910F91FF90EF900C9446
:10433000E105DF91CF911F910F91FF90EF900895CC
:10434000E0917302F0917402309739F022E0DC01C1
:104350002C930480F581E02D099408952091710239
:10436000309172022817390771F09093720280938E
:104370007102E0917302F0917402309721F006808F
:10438000F781E02D0994089520916F023091700219
:104390002817390771F09093700280936F02E091B3
:1043A0007302F0917402309721F00084F185E02DC2
:1043B00009940895FC01329697E080E0915029F02D
:1043C00021912223D9F38F5FF9CF0895662349F015
:1043D000FC01329608962191621729F0E817F90737
:1043E000D1F780E0089581E008959C01FC013296A8
:1043F0009FEF80E04191461789F09F3F19F44111EA
:1044000001C0982F8F5F8630A9F79F3F39F0F901DF
:10441000E90FF11D97FDFA956283089508959C01B7
:104420002A5F3F4FFC014281461301C01282019670
:1044300082179307B9F708950C94F5210C940F2275
:10444000029626E0FC0111922A95E9F70895089555
:104450000C94272283E0809375020C94282281110A
:1044600002C081E001C082E0809375020C94282292
:104470000C942F2281E0809375020C9428220C94D6
:104480003A2208950C9441220C9442220C94412229
:104490000C9441220C9441220E9448220E94501800
:1044A0000E94462280E00E949B1791E0811101C08A
:1044B00090E0892F089508951F920F920FB60F92E2
:1044C00011248F939F93AF93BF93809176028111B4
:1044D00013C080918B0290918C02A0918D02B091BB
:1044E0008E024196A11DB11D80938B0290938C0288
:1044F000A0938D02B0938E02BF91AF919F918F9147
:104500000F900FBE0F901F901895809193028430EA
:1045100031F10E945F081092760220E488E190E079
:104520000FB6F894A895809360000FBE20936000AA
:1045300083B7817F846083BF83B7816083BF7894B2
:10454000889583B78E7F83BF0FB6F894A895809126
:104550006000886180936000109260000FBE089533
:104560000E94C30D0C94630882E084BD93E095BD66
:104570009AEF97BD80936E0008952FB7F8948091BD
:104580008B0290918C02A0918D02B0918E022FBF70
:1045900008952FB7F89460918B0270918C028091EE
:1045A0008D0290918E022FBF08959C014FB7F89411
:1045B00080918B0290918C02A0918D02B0918E021D
:1045C0004FBF821B930B089578941F920F920FB6E2
:1045D0000F9211248F939F93AF93BF9380918B027F
:1045E00090918C02A0918D02B0918E020196A11D36
:1045F000B11D80938B0290938C02A0938D02B09397
:104600008E02BF91AF919F918F910F900FBE0F902F
:104610001F90189581E08093E00080E28093D8009D
:104620001092C9008FE19EE40197F1F700C00000ED
:1046300087E090EBDC0180939C0290939D02A09315
:104640009E02B0939F029CE088E10FB6F894A89573
:10465000809360000FBE90936000FFCF8091850231
:104660000895089522E02093E9002FEF3091E800AB
:10467000215035FD06C035ED3A95F1F700002111C6
:10468000F5CF2091E80025FF0BC040E050E066E048
:1046900070E00E941A268091E8008E778093E800EF
:1046A0000895CF93DF9321E02093E9002FEF30911D
:1046B000E800215035FD06C035ED3A95F1F70000D0
:1046C0002111F5CF2091E80025FF14C0EC0140E056
:1046D00050E068E070E00E941A268091E8008E7732
:1046E0008093E80088E0FE01ADE7B2E001900D9212
:1046F0008A95E1F7DF91CF910895809379027093C5
:104700007B0260937A0280919302843001F582E00B
:104710008093E9008FEF9091E800815095FD06C0ED
:1047200095ED9A95F1F700008111F5CF8091E800A1
:1047300085FF0DC040E050E063E070E089E792E063
:104740000E941A268091E8008E778093E8000895F1
:10475000BC0184E00C947D23BC0183E00C947D2398
:1047600081EB99E00E94E10580919202811109C0DC
:104770000E94AB270E9408288091E2008460809309
:10478000E20008958DEA99E00E94E10510929202FC
:10479000089589EA99E00E94E1050C943F2285EA98
:1047A00099E00E94E10560918F0281E0611101C0F2
:1047B00080E00C942A2281EA99E00E94E105909120
:1047C000930281E0943009F080E060918F020C94B4
:1047D0002F22209178022F5F822F62E30E94B72A56
:1047E000992319F02093780208951092780280910D
:1047F0007C02882371F180919302843041F580918D
:10480000E9008F702091EC00922F917020FD90E8CC
:10481000892B93E09093E9009091EB0090FF14C0F6
:104820009091EE0097FF10C09091E80095FF03C0B3
:104830001092F100F9CF9091E80090FF05C090919F
:10484000E8009E779093E8008F708093E9001092C3
:104850007C02089542E061EC81E00E94242742E25C
:1048600061EC82E00E94242742E261EC83E00E9436
:1048700024279091930281E0943009F080E06091C8
:104880008F020C94382280919502833009F461C024
:1048900030F4813071F0823009F49AC008958A3082
:1048A00009F486C08B3009F46CC0893009F0A8C0C7
:1048B00020C080919402813A09F0A2C08091E80062
:1048C000877F8093E8008091980290919902892BCC
:1048D00021F468E08DE792E003C060E080E090E0C2
:1048E00070E00E9465268091E8008B778093E80055
:1048F000089580919402813209F082C080919802DB
:1049000090919902029708F07BC08091E800877F20
:104910008093E8008091E80082FD05C080919302B9
:104920008111F8CF6DC02091F3008091F20090E0EA
:10493000922B029731F48091F100813011F0863092
:1049400021F48091F100809385028091E8008B77BB
:1049500053C080919402813A09F052C0809198022C
:1049600090919902892B09F04BC08091E800877FD4
:104970008093E8008091E80080FFFCCF80911801CF
:1049800036C0809194028132D9F58091980290913D
:104990009902892BA9F58091E800877F8093E80030
:1049A0000E94592780919602809318010C94C30DA0
:1049B00080919402813221F58091E800877F809375
:1049C000E8000E94592780919702809386020895FB
:1049D00080919402813AA1F48091E800877F8093CE
:1049E000E8008091E80080FFFCCF809186028093F0
:1049F000F1008091E8008E778093E8000C945927AD
:104A000008959FB7F89410927C029FBF90919302F3
:104A1000943009F057C09091E9009F703091EC00FC
:104A2000232F217030FD20E8922B23E02093E90012
:104A30002091EB0020FF43C02091EE0027FF3FC0F4
:104A400020917702222321F02091E80025FF37C032
:104A50001092770226E03091E80035FD15C03091C4
:104A60009302343061F53091EB0035FD28C02150C0
:104A700021F481E08093770222C0EFE9FFE03197D3
:104A8000F1F700C00000E7CF8093F1008091E800CB
:104A900085FD0AC08091E80080FFFCCF8091E8008E
:104AA0008E778093E80006C08FB7F89421E02093BA
:104AB0007C028FBF9F709093E90080E008959F7003
:104AC0009093E9008FEF089584B7877F84BF0FB676
:104AD000F894A8958091600088618093600010929E
:104AE00060000FBE90E080E80FB6F89480936100FC
:104AF000909361000FBE0C943A220E94AB270E9453
:104B00000828E2EEF0E080818460808378940C9441
:104B10009C2A8CE091E00C94462180919302853090
:104B2000C9F48DE999E00E94E105809193028530F6
:104B300079F40E948522809191028823B1F30E942A
:104B40004C22882391F30E9404260E94C30DEDCFCE
:104B50000C94B022089508950C94AE25292F332784
:104B600023303105C9F060F42130310581F0223065
:104B7000310509F041C08BE590E02BEE39E040C0F3
:104B800021323105E1F02232310531F135C082E1C7
:104B900090E026E43AE034C099278130910549F04D
:104BA00028F0029749F5E5EBF9E005C0E7EEF9E0FA
:104BB00002C0EDECF9E0849190E09F0121C06330E8
:104BC0007105D0F4660F771FFB01E951FE4F20817C
:104BD000318189E090E014C06330710568F4FB0115
:104BE000EE0FFF1FEF51FE4F20813181FB01E2529A
:104BF000FE4F808190E004C080E090E020E030E053
:104C0000FA0131832083089580E189BD82E189BD65
:104C100009B400FEFDCF8091D8008F7D8093D8002D
:104C20008091E00082608093E0008091E00081FD4F
:104C3000FCCF0895CF92DF92EF92FF920F931F93D4
:104C4000CF93DF93EC018B017A010E9478278111C9
:104C500033C0E114F10439F0F70180819181081B20
:104C6000190BC80FD91FC12CD12C0115110519F131
:104C70008091E80085FD16C08091E8008E778093D2
:104C8000E800E114F10449F0F70180819181C80E38
:104C9000D91ED182C08285E00FC00E947827882368
:104CA00021F30AC089918093F10001501109FFEFAF
:104CB000CF1ADF0ADACF80E0DF91CF911F910F91F9
:104CC000FF90EF90DF90CF90089520919A0230915D
:104CD0009B022617370748F06115710539F42091BA
:104CE000E8002E772093E80001C0B901FC0120E024
:104CF0006115710579F1809193028823F1F1853076
:104D0000F1F18091E80083FD3CC08091E80082FDD4
:104D10002EC08091E80080FFEBCF2091F3008091BE
:104D2000F20090E0922B6115710551F088309105E9
:104D300038F421912093F100615071090196F3CF6D
:104D400021E0089709F020E08091E8008E778093B9
:104D5000E800CECF2111CFCF0AC0809193028823E3
:104D600061F0853061F08091E80083FD0AC0809198
:104D7000E80082FFF2CF80E0089582E0089583E0AA
:104D8000089581E0089520919A0230919B022617A0
:104D9000370748F06115710539F42091E8002E7746
:104DA0002093E80001C0B901FC0120E06115710504
:104DB00091F180919302882309F440C0853009F471
:104DC0003FC08091E80083FD3DC08091E80082FDF6
:104DD0002FC08091E80080FFE9CF2091F3008091FF
:104DE000F20090E0922B6115710559F08830910521
:104DF00040F424912093F10031966150710901969D
:104E0000F2CF21E0089709F020E08091E8008E774A
:104E10008093E800CBCF2111CCCF0AC080919302C0
:104E2000882361F0853061F08091E80083FD0AC03D
:104E30008091E80082FFF2CF80E0089582E008953B
:104E400083E0089581E00895982F973068F5909356
:104E5000E900981739F07091EC002091ED00509125
:104E6000F00003C0242F762F50E021FD02C09F5F89
:104E7000ECCF3091EB003E7F3093EB003091ED00B2
:104E80003D7F3093ED003091EB0031603093EB00CB
:104E90007093EC002093ED005093F0002091EE0011
:104EA00027FDE5CF80E008958F708093E90081E0D1
:104EB00008958091940287FF11C08091E80082FDDF
:104EC00005C0809193028111F8CF11C08091E80054
:104ED0008B770BC080919302882349F08091E80082
:104EE00080FFF8CF8091E8008E778093E8000895E6
:104EF0002091E4003091E50095E64091EC00842F8C
:104F0000817040FF23C08091E80080FD1DC080912A
:104F10009302882399F0853099F08091EB0085FD0C
:104F200011C04091E4005091E5002417350729F3A2
:104F3000915011F09A01E1CF84E0089582E0089544
:104F400083E0089581E0089580E008954091E800AD
:104F500042FFDDCF08950E9419280E942128E0EE2B
:104F6000F0E0808181608083E8EDF0E080818F77E0
:104F7000808319BCA7EDB0E08C918E7F8C938081EB
:104F80008F7E80831092920208950F931F93CF9388
:104F9000DF930E9419280E942128C8EDD0E0888163
:104FA0008F77888388818068888388818F7D8883D4
:104FB00019BC1092930210928F02109291021092DB
:104FC000900200EE10E0F80180818B7F8083888161
:104FD0008160888342E060E080E00E942427E1EE67
:104FE000F0E080818E7F8083E2EEF0E0808181605E
:104FF0008083808188608083F80180818E7F8083B8
:10500000888180618883DF91CF911F910F910895EE
:10501000E8EDF0E080818F7E8083E7EDF0E0808135
:105020008160808384E082BF81E0809392020C944F
:10503000C527E8EDF0E080818E7F80831092E2004A
:1050400008951092DA001092E10008951F920F92D5
:105050000FB60F9211242F933F934F935F936F934B
:105060007F938F939F93AF93BF93EF93FF93809121
:10507000E10082FF0BC08091E20082FF07C08091B7
:10508000E1008B7F8093E1000E94E9238091DA00A8
:1050900080FF1FC08091D80080FF1BC08091DA0084
:1050A0008E7F8093DA008091D90080FF0DC080E16F
:1050B00089BD82E189BD09B400FEFDCF81E0809306
:1050C00093020E94B02305C019BC109293020E9463
:1050D000C2238091E10080FF19C08091E20080FF2F
:1050E00015C08091E2008E7F8093E2008091E20003
:1050F00080618093E2008091D80080628093D80024
:1051000019BC85E0809393020E94CF238091E10037
:1051100084FF30C08091E20084FF2CC080E189BD13
:1051200082E189BD09B400FEFDCF8091D8008F7D5A
:105130008093D8008091E1008F7E8093E100809180
:10514000E2008F7E8093E2008091E2008160809394
:10515000E20080918F02882311F084E007C08091E3
:10516000E30087FD02C081E001C083E080939302E9
:105170000E94DB238091E10083FF29C08091E2003F
:1051800083FF25C08091E100877F8093E10082E06A
:105190008093930210928F028091E1008E7F809322
:1051A000E1008091E2008E7F8093E2008091E20036
:1051B00080618093E20042E060E080E00E9424276A
:1051C0008091F00088608093F0000E94C923FF91D5
:1051D000EF91BF91AF919F918F917F916F915F916F
:1051E0004F913F912F910F900FBE0F901F901895E8
:1051F0001F920F920FB60F9211242F933F934F934C
:105200005F936F937F938F939F93AF93BF93CF934E
:10521000DF93EF93FF93C091E900CF708091EC0092
:10522000D82FD17080FDD0E81092E9008091F00075
:10523000877F8093F00078940E943C291092E900C7
:105240008091F00088608093F000CD2BCF70C093E8
:10525000E900FF91EF91DF91CF91BF91AF919F91C5
:105260008F917F916F915F914F913F912F910F900F
:105270000FBE0F901F9018951F93CF93DF93CDB75C
:10528000DEB7AA970FB6F894DEBF0FBECDBFE4E934
:10529000F2E08091F100819322E0EC39F207C9F746
:1052A0000E9443248091E80083FF2EC180919402E4
:1052B00090919502492F50E04A30510508F024C1E1
:1052C000FA01EE59FF4F0C94D72A803821F082382A
:1052D00009F01AC108C0809190029091910299231F
:1052E00089F082600FC0809198028F70873008F03B
:1052F0000BC18093E9008091EB0085FB882780F942
:105300001092E9009091E800977F9093E8008093D5
:10531000F1001092F100D1C0282F2D7F09F0F4C0C8
:10532000882319F0823061F0EFC0809196028130BD
:1053300009F0EAC0933009F080E0809391022EC01A
:105340008091960281112AC0809198028F702FEF70
:10535000280F263008F0D8C08093E9002091EB0098
:1053600020FF1CC0933021F48091EB00806214C0B8
:105370009091EB0090619093EB0021E030E0A90167
:1053800002C0440F551F8A95E2F74093EA0010923D
:10539000EA008091EB0088608093EB001092E900B6
:1053A0008091E800877F8093E8000E945927ACC075
:1053B0008111AAC0109196021F778091E300807836
:1053C000812B8093E3008091E800877F8093E80041
:1053D0000E9459278091E80080FFFCCF8091E30074
:1053E00080688093E300111102C082E001C083E075
:1053F0008093930289C08058823008F085C08091E4
:105400009602909197028C3D53E0950779F583E0E1
:105410008A838AE289834FB7F894DE01139620E0ED
:105420003EE051E2E32FF0E050935700E49120FF7B
:1054300003C0E295EF703F5FEF708E2F90E0EA308F
:1054400010F0C79601C0C0968D939D932F5F2431B5
:1054500049F74FBF8091E800877F8093E8006AE2B8
:1054600070E0CE0101960E94652616C060919802F8
:1054700070919902AE014F5F5F4F0E94AC25BC0155
:10548000892B09F441C09091E800977F9093E80040
:1054900089819A810E94C3268091E8008B7780934E
:1054A000E80032C0803881F58091E800877F8093E2
:1054B000E80080918F028093F1008091E8008E7760
:1054C00072CF811121C08091960290919702992705
:1054D0000297D4F48091E800877F8093E800809160
:1054E000960280938F020E94592780918F0281112A
:1054F00006C08091E30087FD02C081E001C084E026
:10550000809393020E942A248091E80083FF0AC0BE
:105510008091E800877F8093E8008091EB008062B3
:105520008093EB00AA960FB6F894DEBF0FBECDBFF6
:10553000DF91CF911F910895CF938091930288239B
:10554000A1F0C091E900CF709091EC00892F81709B
:1055500090FD80E8C82B1092E9008091E80083FD5F
:105560000E943C29CF70C093E900CF910895991B08
:1055700079E004C0991F961708F0961B881F7A954A
:10558000C9F78095089597FB072E16F4009407D06D
:1055900077FD09D00E94DD2A07FC05D03EF49095E6
:1055A00081959F4F0895709561957F4F0895EE0FF7
:1055B000FF1F0590F491E02D0994AA1BBB1B51E13C
:1055C00007C0AA1FBB1FA617B70710F0A61BB70B73
:1055D000881F991F5A95A9F780959095BC01CD0118
:1055E0000895FB01DC0104C08D910190801921F424
:1055F00041505040C8F7881B990B0895F999FECF88
:1056000092BD81BDF89A992780B50895A8E1B0E0D0
:1056100042E050E00C94322B262FF999FECF92BD38
:1056200081BDF89A019700B4021639F01FBA20BD67
:105630000FB6F894FA9AF99A0FBE08950396272F99
:105640000E940D2B0E940C2B252F0E940D2B242F26
:105650000C940D2B0196272F0E940D2B0C940C2BD4
:10566000DC01CB01FC01F999FECF06C0F2BDE1BD22
:10567000F89A319600B40D9241505040B8F7089511
:04568000F894FFCFCC
:10568400C8004102280850011E0A14012E23512388
:105694003223AC23A823312301E200E900EA00B558
:1056A40000B600B700CD008301CC008A01920194BA
:1056B400012102230224022502260227022A02B320
:1056C40000B4006F007000818283E200E900EA0008
:1056D400B500B600B700CD008301CC008A01920169
:1056E40094012102230224022502260227022A020F
:1056F400B300B4006F007000818283F7F6F5F4F113
:10570400F03F3F3F006D6B5F64656C6179006D6BCA
:105714005F696E74657276616C006D6B5F6D617844
:105724005F7370656564006D6B5F74696D655F744C
:105734006F5F6D6178006D6B5F776865656C5F6D39
:1057440061785F7370656564006D6B5F776865652C
:105754006C5F74696D655F746F5F6D617800407B29
:0E57640022F50A7A0A580AFD09160A2F0A00D1
:00000001FF
